:10000000830100308A002D288C0003088301C8007A
:100010000B1D2728DF30831281008E08031D8E03FD
:100020008F08031D8F039508031926281508033927
:10003000031D25280D1C1E2886141F2886100D1050
:1000400014180D1403148312940C95030B118312CE
:10005000480883008C0E0C0E09000E3084003930E5
:100060003A200D3084000E303A2083012329040603
:0C0070008001840A0406031D37280034B8
:10009A009A3083128F008F080319080050281430F1
:1000AA0083128E008E080319080057288312B7009E
:1000BA008900831608148312080808008312B10005
:1000CA00310E0F39B200782031080F39B200782882
:1000DA008312B4009508031D6F280D10340894008C
:1000EA003430950008008312B3000A303302031833
:1000FA008028303081283730B30733086D288312BF
:10010A00B2008C28B20A32035B206D208312B1033D
:10011A00310F8728080083120510B801B71F9728E6
:10012A00851498288510831205150310B60DB70D8E
:10013A0005118510B80A10303802031C93280514DB
:10014A00080028308312AF00AE012E08B900031050
:10015A00B90D0310390D163EB0002F0883124F2235
:10016A000430AF07AE0A06302E0203180800AA2888
:10017A008312861495018E018F0193019001FF303D
:10018A00910001308500183083168500FD30860005
:10019A00811381128B16DF30831281008B170800BE
:1001AA008312B4000430B5003008B60035083407AD
:1001BA00B90039038312EE203108B0003208B100C9
:1001CA003308B200B301B50301303502031C08003D
:1001DA00D9288312B70083168818F12883123708A2
:1001EA0089003608880003108B1B03148B138316AF
:1001FA00081555308900AA30890088140811031897
:10020A008B1783120800831205140511B601F83002
:10021A00B7009020B601B030B7009020B601403048
:10022A00B7009020B6011830B7009020B601093007
:10023A00B7009020B601C030B70090288312BD20C5
:10024A00082105081839031D2D29B6012730EE208B
:10025A002030B10000308420942142210508183949
:10026A00031D3F294D20930A06301302031C32292D
:10027A0093013229AB22C4213F298312B101B10A69
:10028A00203084201308303E6D2020306D20130862
:10029A00B9000310B90D0310390D163EAF00043032
:1002AA00B00030082F07B900390384000008632022
:1002BA00B003013030020318562900220230B1007F
:1002CA001E30842828308312AF00AE012E08B900F0
:1002DA000310B90D0310390D163E84000008B90049
:1002EA00840A0008BA00840A0008BB00840A0008CD
:1002FA00BC003908B0003A08B1003B08B2003C081B
:10030A00B3002F088312D5200430AF07AE0A063097
:10031A002E02031C6B29B601B60A2730EE282730B5
:10032A0083125B200038031DA628723096004B30DA
:10033A0097005B309800990190309A0008309B0032
:10034A008A309C009D01CD309E007D309F00AF30E9
:10035A00A000A1015830A2001430A3009330A400D9
:10036A00A5012430A6006430A700C730A800A9015F
:10037A00AA018530AB00CF30AC00AD0167298312EA
:10038A000608AE00FC3990000630930010087C3A4B
:10039A00031993011008BC3A031DD5299301930A46
:1003AA001008DC3A031DDB29023093001008EC3AEE
:1003BA00031DE129033093001008F43A031DE729CD
:1003CA00043093001008F83A031DED290530930014
:1003DA001308063A0319F929130812060319F92909
:1003EA0083124221130892001308063A031D0800DB
:0603FA0012089300080048
:1004000083121308B9000310B90D0310390D163EFD
:1004100084000008B900840A0008BA00840A0008B1
:10042000BB00840A0008BC009E239530BD00BF308D
:10043000BE00D630BF004230C000B023632339086D
:10044000B2003A08B3003B08B4003C08B5003230B3
:10045000B100840000300004B6003030B7008312D1
:100460009020310A840000300004B6002130B7002B
:1004700090203108023E840000300004B600323083
:10048000B70090203108033E840000300004B6001D
:100490002330B7009020B6015030B7009028831267
:1004A000B100B201300884000008B900840A0008D5
:1004B000BA00840A0008BB00840A0008BC003B089C
:1004C000BC003A08BB003908BA00B9013008840002
:1004D00039088000840A3A088000840A3B088000BA
:1004E000840A3C088000300884000008B900840AAF
:1004F0000008BA00840A0008BB00840A0008BC0097
:1005000039088312B3003A08B4003B08B5003C0830
:10051000B600310832075B20B900BA01BB01BC014B
:100520003308B9043408BA043508BB043608BC04DF
:100530003008840039088000840A3A088000840A60
:100540003B088000840A3C088000B20A0430320272
:1005500003180800522A83120508183911060319D6
:10056000062B0508183991004D2005081839110689
:10057000031D4D281308063A0319022B1108103ADF
:10058000031DE02A1308B9000310B90D0310390D3B
:10059000163E840005308007840A00300318013EAF
:1005A000031D8007840A00300318013E031D8007E5
:1005B000840A00300318013E80078312422167211C
:1005C0001108083A031D022B1308B9000310B90DD6
:1005D0000310390D163E8400FB308007840AFF307B
:1005E0000318013E031D8007840AFF300318013EF3
:1005F000031D8007840AFF300318013E8007831221
:10060000422167210508183991004D281108183A30
:1006100003190800BA2A8312C7013B0D3C0DC5001F
:1006200045080319172BC70DBC01BB170800B901FA
:10063000BA01BB01BC010034C7103F0D400DC6001C
:1006400046080319282B0318C714C001BF17080058
:10065000C601BD01BE01BF01C00108004508031964
:10066000172BBB13C70C450CBC000318BB17A12BE1
:10067000C50803195E2B3C0803194E2B3C030319D4
:10068000B90A0319BA0A0319BB0A0319BC0A0310F1
:10069000BC0CBB0CBA0CB90CC50A382B39083A048F
:1006A0003B043C0403195E2BBB1B2E2BC503031913
:1006B0005E2B0310B90DBA0DBB0D542BB901BA0155
:1006C000BB01BC01A12B84010B238230C507C51BD4
:1006D000172BE830C507C51B7E2B203045020318B9
:1006E000172BC50803197B2BC5030310B90DBA0DD1
:1006F000BB0DBC0D712B4718862308000310BC0CE2
:10070000BB0CBA0CB90CC50F7E2B7B2B0310FF3032
:10071000B907B909031CBA07BA09031CBB07BB090F
:10072000031CBC07BC0908008312C701BC1F9A2B1D
:10073000471486239630C5008401382B8312C701E5
:100740009A2B8408031900343C08800084033B087A
:10075000800084033A088000840339088000003454
:1007600084010B231C23C101C201C301C401073052
:10077000C0000310BF0CBE0CBD0C031CCE2B3908EF
:10078000C1073A0803183A0FC2073B0803183B0F8A
:10079000C3073C0803183C0AC4070310B90DBA0D7F
:1007A000BB0DBC0DC00BB92B1130C000DC2B0310EE
:1007B000C40CC30CC20CC10C0310BF0CBE0CBD0C8E
:1007C000031CF02B3908C1073A0803183A0FC20777
:1007D0003B0803183B0FC3073C0803183C0AC40737
:1007E000C00BD72B7A304607C507470CC706410810
:1007F000B9004208BA004308BB004408BC00382BCB
:02400E00F13F80
:104200005000690063004400440053002D00360054
:104210004600200031002E0031002000280043001D
:10422000290020003200300030003400200042001D
:104230002E00560045004C004C0045000D000A00C1
:1042400046002D002D002D002D002D002D0000001A
:10425000000000000000000000000000000000005E
:10426000000000000000000000000000000000004E
:10427000000000000000000000000000000000003E
:00000001FF
